 dt_shmem

 Timestamp is ffffffff (Sun Feb  7 06:28:15 2106)

 Preferred load address is 10000000

 Start         Length     Name                   Class
 0001:00000000 0000311eH .text$mn                CODE
 0002:00000000 000000e8H .idata$5                DATA
 0002:000000e8 00000004H .00cfg                  DATA
 0002:000000ec 00000004H .CRT$XCA                DATA
 0002:000000f0 00000004H .CRT$XCZ                DATA
 0002:000000f4 00000004H .CRT$XIA                DATA
 0002:000000f8 00000004H .CRT$XIZ                DATA
 0002:000000fc 00000004H .CRT$XPA                DATA
 0002:00000100 00000004H .CRT$XPZ                DATA
 0002:00000104 00000004H .CRT$XTA                DATA
 0002:00000108 00000008H .CRT$XTZ                DATA
 0002:0000010c 00000000H .gfids$y                DATA
 0002:00000110 00000728H .rdata                  DATA
 0002:00000838 00000004H .rdata$sxdata           DATA
 0002:0000083c 00000288H .rdata$zzzdbg           DATA
 0002:00000ac4 00000004H .rtc$IAA                DATA
 0002:00000ac8 00000004H .rtc$IZZ                DATA
 0002:00000acc 00000004H .rtc$TAA                DATA
 0002:00000ad0 00000008H .rtc$TZZ                DATA
 0002:00000ad8 00000088H .xdata$x                DATA
 0002:00000b60 00000388H .edata                  DATA
 0002:00000ee8 00000078H .idata$2                DATA
 0002:00000f60 00000014H .idata$3                DATA
 0002:00000f74 000000e8H .idata$4                DATA
 0002:0000105c 00000466H .idata$6                DATA
 0003:00000000 00000028H .data                   DATA
 0003:00000028 000003ccH .bss                    DATA
 0004:00000000 00000060H .rsrc$01                DATA
 0004:00000060 00000328H .rsrc$02                DATA

  Address         Publics by Value              Rva+Base       Lib:Object

 0000:00000000       ___dynamic_value_reloc_table 00000000     <absolute>
 0000:00000000       ___hybrid_code_map         00000000     <absolute>
 0000:00000000       ___guard_fids_table        00000000     <absolute>
 0000:00000000       ___hybrid_auxiliary_iat    00000000     <absolute>
 0000:00000000       ___guard_iat_table         00000000     <absolute>
 0000:00000000       ___arm64x_redirection_metadata_count 00000000     <absolute>
 0000:00000000       ___guard_longjmp_count     00000000     <absolute>
 0000:00000000       ___arm64x_native_entrypoint 00000000     <absolute>
 0000:00000000       ___hybrid_code_map_count   00000000     <absolute>
 0000:00000000       ___guard_longjmp_table     00000000     <absolute>
 0000:00000000       ___guard_fids_count        00000000     <absolute>
 0000:00000000       ___x64_code_ranges_to_entry_points 00000000     <absolute>
 0000:00000000       ___volatile_metadata       00000000     <absolute>
 0000:00000000       ___enclave_config          00000000     <absolute>
 0000:00000000       ___guard_eh_cont_count     00000000     <absolute>
 0000:00000000       ___guard_iat_count         00000000     <absolute>
 0000:00000000       ___arm64x_redirection_metadata 00000000     <absolute>
 0000:00000000       ___AbsoluteZero            00000000     <absolute>
 0000:00000000       ___guard_eh_cont_table     00000000     <absolute>
 0000:00000000       ___arm64x_extra_rfe_table_size 00000000     <absolute>
 0000:00000000       ___arm64x_extra_rfe_table  00000000     <absolute>
 0000:00000000       ___x64_code_ranges_to_entry_points_count 00000000     <absolute>
 0000:00000001       ___safe_se_handler_count   00000001     <absolute>
 0000:00000100       ___guard_flags             00000100     <absolute>
 0000:00000000       ___ImageBase               10000000     <linker-defined>
 0001:00000000       _Java_com_sun_tools_jdi_SharedMemoryConnection_close0@16 10001000 f   SharedMemoryConnection.obj
 0001:0000000d       _Java_com_sun_tools_jdi_SharedMemoryConnection_receiveByte0@16 1000100d f   SharedMemoryConnection.obj
 0001:0000003f       _Java_com_sun_tools_jdi_SharedMemoryConnection_receivePacket0@16 1000103f f   SharedMemoryConnection.obj
 0001:00000094       _Java_com_sun_tools_jdi_SharedMemoryConnection_sendByte0@20 10001094 f   SharedMemoryConnection.obj
 0001:000000bc       _Java_com_sun_tools_jdi_SharedMemoryConnection_sendPacket0@20 100010bc f   SharedMemoryConnection.obj
 0001:000003c1       _Java_com_sun_tools_jdi_SharedMemoryTransportService_accept0@24 100013c1 f   SharedMemoryTransport.obj
 0001:00000418       _Java_com_sun_tools_jdi_SharedMemoryTransportService_attach0@20 10001418 f   SharedMemoryTransport.obj
 0001:00000492       _Java_com_sun_tools_jdi_SharedMemoryTransportService_initialize@8 10001492 f   SharedMemoryTransport.obj
 0001:000004dc       _Java_com_sun_tools_jdi_SharedMemoryTransportService_name@16 100014dc f   SharedMemoryTransport.obj
 0001:00000543       _Java_com_sun_tools_jdi_SharedMemoryTransportService_startListening0@12 10001543 f   SharedMemoryTransport.obj
 0001:000005c2       _Java_com_sun_tools_jdi_SharedMemoryTransportService_stopListening0@16 100015c2 f   SharedMemoryTransport.obj
 0001:000005cf       ___local_stdio_printf_options 100015cf f i SharedMemoryTransport.obj
 0001:000005d5       __vsnprintf_l              100015d5 f i SharedMemoryTransport.obj
 0001:00000608       _sprintf                   10001608 f i SharedMemoryTransport.obj
 0001:00000622       _throwException            10001622 f   SharedMemoryTransport.obj
 0001:0000064c       _throwShmemException       1000164c f   SharedMemoryTransport.obj
 0001:0000075e       _jdwpTransport_OnLoad@16   1000175e f   shmemBack.obj
 0001:00000c37       __vfprintf_l               10001c37 f i shmemBase.obj
 0001:0000140f       _exitTransportWithError    1000240f f   shmemBase.obj
 0001:000014a5       _fprintf                   100024a5 f i shmemBase.obj
 0001:000019fd       _shmemBase_accept          100029fd f   shmemBase.obj
 0001:00001a9f       _shmemBase_attach          10002a9f f   shmemBase.obj
 0001:00001b56       _shmemBase_closeConnection 10002b56 f   shmemBase.obj
 0001:00001b60       _shmemBase_closeTransport  10002b60 f   shmemBase.obj
 0001:00001b6a       _shmemBase_getlasterror    10002b6a f   shmemBase.obj
 0001:00001b8d       _shmemBase_initialize      10002b8d f   shmemBase.obj
 0001:00001bac       _shmemBase_listen          10002bac f   shmemBase.obj
 0001:00001bd4       _shmemBase_name            10002bd4 f   shmemBase.obj
 0001:00001be1       _shmemBase_receiveByte     10002be1 f   shmemBase.obj
 0001:00001cb6       _shmemBase_receivePacket   10002cb6 f   shmemBase.obj
 0001:00001de9       _shmemBase_sendByte        10002de9 f   shmemBase.obj
 0001:00001ec4       _shmemBase_sendPacket      10002ec4 f   shmemBase.obj
 0001:000020d5       _sysProcessClose           100030d5 f   shmem_md.obj
 0001:000020d5       _sysEventClose             100030d5 f   shmem_md.obj
 0001:000020d5       _sysIPMutexClose           100030d5 f   shmem_md.obj
 0001:000020e7       _sysEventCreate            100030e7 f   shmem_md.obj
 0001:0000212f       _sysEventOpen              1000312f f   shmem_md.obj
 0001:00002153       _sysEventSignal            10003153 f   shmem_md.obj
 0001:00002165       _sysEventWait              10003165 f   shmem_md.obj
 0001:000021b6       _sysGetLastError           100031b6 f   shmem_md.obj
 0001:00002210       _sysIPMutexCreate          10003210 f   shmem_md.obj
 0001:0000224d       _sysIPMutexEnter           1000324d f   shmem_md.obj
 0001:0000227b       _sysIPMutexExit            1000327b f   shmem_md.obj
 0001:0000228d       _sysIPMutexOpen            1000328d f   shmem_md.obj
 0001:000022b1       _sysProcessGetID           100032b1 f   shmem_md.obj
 0001:000022ba       _sysProcessOpen            100032ba f   shmem_md.obj
 0001:000022de       _sysSharedMemClose         100032de f   shmem_md.obj
 0001:00002308       _sysSharedMemCreate        10003308 f   shmem_md.obj
 0001:0000236c       _sysSharedMemOpen          1000336c f   shmem_md.obj
 0001:000023b4       _sysSleep                  100033b4 f   shmem_md.obj
 0001:000023bf       _sysTlsAlloc               100033bf f   shmem_md.obj
 0001:000023c5       _sysTlsGet                 100033c5 f   shmem_md.obj
 0001:000023d0       _sysTlsPut                 100033d0 f   shmem_md.obj
 0001:000023df       @__security_check_cookie@4 100033df f   MSVCRT:secchk.obj
 0001:00002730       __DllMainCRTStartup@12     10003730 f   MSVCRT:dll_dllmain.obj
 0001:00002753       ___raise_securityfailure   10003753 f   MSVCRT:gs_report.obj
 0001:0000277b       ___report_gsfailure        1000377b f   MSVCRT:gs_report.obj
 0001:000028c1       ___security_init_cookie    100038c1 f   MSVCRT:gs_support.obj
 0001:0000290c       _DllMain@12                1000390c f   MSVCRT:dll_dllmain_stub.obj
 0001:0000292e       ?__scrt_initialize_type_info@@YAXXZ 1000392e f   MSVCRT:tncleanup.obj
 0001:0000293a       ?__scrt_uninitialize_type_info@@YAXXZ 1000393a f   MSVCRT:tncleanup.obj
 0001:00002946       ___local_stdio_scanf_options 10003946 f i MSVCRT:default_local_stdio_options.obj
 0001:0000294c       ___scrt_initialize_default_local_stdio_options 1000394c f   MSVCRT:default_local_stdio_options.obj
 0001:000029ad       ___scrt_acquire_startup_lock 100039ad f   MSVCRT:utility.obj
 0001:000029df       ___scrt_dllmain_after_initialize_c 100039df f   MSVCRT:utility.obj
 0001:00002a0a       ___scrt_dllmain_before_initialize_c 10003a0a f   MSVCRT:utility.obj
 0001:00002a18       ___scrt_dllmain_crt_thread_attach 10003a18 f   MSVCRT:utility.obj
 0001:00002a37       ___scrt_dllmain_crt_thread_detach 10003a37 f   MSVCRT:utility.obj
 0001:00002a44       ___scrt_dllmain_exception_filter 10003a44 f   MSVCRT:utility.obj
 0001:00002a78       ___scrt_dllmain_uninitialize_c 10003a78 f   MSVCRT:utility.obj
 0001:00002a9b       ___scrt_dllmain_uninitialize_critical 10003a9b f   MSVCRT:utility.obj
 0001:00002aa8       ___scrt_initialize_crt     10003aa8 f   MSVCRT:utility.obj
 0001:00002ae1       ___scrt_initialize_onexit_tables 10003ae1 f   MSVCRT:utility.obj
 0001:00002b68       ___scrt_is_nonwritable_in_current_image 10003b68 f   MSVCRT:utility.obj
 0001:00002bfc       ___scrt_release_startup_lock 10003bfc f   MSVCRT:utility.obj
 0001:00002c19       ___scrt_uninitialize_crt   10003c19 f   MSVCRT:utility.obj
 0001:00002c41       ___scrt_get_dyn_tls_init_callback 10003c41 f   MSVCRT:dyn_tls_init.obj
 0001:00002c47       ___scrt_fastfail           10003c47 f   MSVCRT:utility_desktop.obj
 0001:00002d61       __crt_debugger_hook        10003d61 f   MSVCRT:utility_desktop.obj
 0001:00002d69       __RTC_Initialize           10003d69 f   MSVCRT:initsect.obj
 0001:00002d95       __RTC_Terminate            10003d95 f   MSVCRT:initsect.obj
 0001:00002dd0       __SEH_prolog4              10003dd0 f   MSVCRT:sehprolg4.obj
 0001:00002e14       __SEH_epilog4              10003e14 f   MSVCRT:sehprolg4.obj
 0001:00002e28       __except_handler4          10003e28 f   MSVCRT:chandler4gs.obj
 0001:00002e57       @_guard_check_icall_nop@4  10003e57 f i MSVCRT:guard_support.obj
 0001:00002e5a       ___isa_available_init      10003e5a f   MSVCRT:cpu_disp.obj
 0001:0000302a       __get_startup_argv_mode    1000402a f   MSVCRT:argv_mode.obj
 0001:0000302e       ___scrt_is_ucrt_dll_in_use 1000402e f   MSVCRT:ucrt_detection.obj
 0001:0000303a       _IsProcessorFeaturePresent@4 1000403a f   kernel32:KERNEL32.dll
 0001:00003040       _memset                    10004040 f   vcruntime:VCRUNTIME140.dll
 0001:00003046       _memcpy                    10004046 f   vcruntime:VCRUNTIME140.dll
 0001:0000304c       ___std_type_info_destroy_list 1000404c f   vcruntime:VCRUNTIME140.dll
 0001:00003052       __except_handler4_common   10004052 f   vcruntime:VCRUNTIME140.dll
 0001:00003058       _free                      10004058 f   ucrt:api-ms-win-crt-heap-l1-1-0.dll
 0001:0000305e       _strcat                    1000405e f   ucrt:api-ms-win-crt-string-l1-1-0.dll
 0001:00003064       _strcpy                    10004064 f   ucrt:api-ms-win-crt-string-l1-1-0.dll
 0001:0000306a       _strlen                    1000406a f   ucrt:api-ms-win-crt-string-l1-1-0.dll
 0001:00003070       __initterm                 10004070 f   ucrt:api-ms-win-crt-runtime-l1-1-0.dll
 0001:00003076       __initterm_e               10004076 f   ucrt:api-ms-win-crt-runtime-l1-1-0.dll
 0001:0000307c       __seh_filter_dll           1000407c f   ucrt:api-ms-win-crt-runtime-l1-1-0.dll
 0001:00003082       __configure_narrow_argv    10004082 f   ucrt:api-ms-win-crt-runtime-l1-1-0.dll
 0001:00003088       __initialize_narrow_environment 10004088 f   ucrt:api-ms-win-crt-runtime-l1-1-0.dll
 0001:0000308e       __initialize_onexit_table  1000408e f   ucrt:api-ms-win-crt-runtime-l1-1-0.dll
 0001:00003094       __execute_onexit_table     10004094 f   ucrt:api-ms-win-crt-runtime-l1-1-0.dll
 0001:0000309a       __cexit                    1000409a f   ucrt:api-ms-win-crt-runtime-l1-1-0.dll
 0001:000030a0       ___vcrt_initialize         100040a0 f   MSVCRT:ucrt_stubs.obj
 0001:000030a0       ___scrt_stub_for_acrt_initialize 100040a0 f   MSVCRT:ucrt_stubs.obj
 0001:000030a0       ___vcrt_thread_detach      100040a0 f   MSVCRT:ucrt_stubs.obj
 0001:000030a0       ___scrt_stub_for_acrt_thread_attach 100040a0 f   MSVCRT:ucrt_stubs.obj
 0001:000030a0       ___acrt_initialize         100040a0 f   MSVCRT:ucrt_stubs.obj
 0001:000030a0       ___vcrt_thread_attach      100040a0 f   MSVCRT:ucrt_stubs.obj
 0001:000030a0       ___scrt_stub_for_acrt_thread_detach 100040a0 f   MSVCRT:ucrt_stubs.obj
 0001:000030a0       ___vcrt_uninitialize_critical 100040a0 f   MSVCRT:ucrt_stubs.obj
 0001:000030a0       ___acrt_uninitialize_critical 100040a0 f   MSVCRT:ucrt_stubs.obj
 0001:000030a0       ___acrt_thread_attach      100040a0 f   MSVCRT:ucrt_stubs.obj
 0001:000030a0       ___acrt_uninitialize       100040a0 f   MSVCRT:ucrt_stubs.obj
 0001:000030a0       ___scrt_stub_for_acrt_uninitialize_critical 100040a0 f   MSVCRT:ucrt_stubs.obj
 0001:000030a0       ___scrt_stub_for_acrt_uninitialize 100040a0 f   MSVCRT:ucrt_stubs.obj
 0001:000030a0       ___acrt_thread_detach      100040a0 f   MSVCRT:ucrt_stubs.obj
 0001:000030a0       ___vcrt_uninitialize       100040a0 f   MSVCRT:ucrt_stubs.obj
 0001:000030a3       ___scrt_stub_for_is_c_termination_complete 100040a3 f   MSVCRT:ucrt_stubs.obj
 0001:000030a3       __is_c_termination_complete 100040a3 f   MSVCRT:ucrt_stubs.obj
 0001:000030a6       __filter_x86_sse2_floating_point_exception_default 100040a6 f   MSVCRT:x86_exception_filter.obj
 0001:000030a6       __filter_x86_sse2_floating_point_exception 100040a6 f   MSVCRT:x86_exception_filter.obj
 0002:00000000       __imp__CloseHandle@4       10005000     kernel32:KERNEL32.dll
 0002:00000004       __imp__GetLastError@0      10005004     kernel32:KERNEL32.dll
 0002:00000008       __imp__SetEvent@4          10005008     kernel32:KERNEL32.dll
 0002:0000000c       __imp__ReleaseMutex@4      1000500c     kernel32:KERNEL32.dll
 0002:00000010       __imp__CreateMutexA@12     10005010     kernel32:KERNEL32.dll
 0002:00000014       __imp__CreateEventA@16     10005014     kernel32:KERNEL32.dll
 0002:00000018       __imp__OpenEventA@12       10005018     kernel32:KERNEL32.dll
 0002:0000001c       __imp__Sleep@4             1000501c     kernel32:KERNEL32.dll
 0002:00000020       __imp__WaitForMultipleObjects@16 10005020     kernel32:KERNEL32.dll
 0002:00000024       __imp__GetCurrentProcessId@0 10005024     kernel32:KERNEL32.dll
 0002:00000028       __imp__TlsAlloc@0          10005028     kernel32:KERNEL32.dll
 0002:0000002c       __imp__TlsGetValue@4       1000502c     kernel32:KERNEL32.dll
 0002:00000030       __imp__TlsSetValue@8       10005030     kernel32:KERNEL32.dll
 0002:00000034       __imp__OpenProcess@12      10005034     kernel32:KERNEL32.dll
 0002:00000038       __imp__MapViewOfFile@20    10005038     kernel32:KERNEL32.dll
 0002:0000003c       __imp__UnmapViewOfFile@4   1000503c     kernel32:KERNEL32.dll
 0002:00000040       __imp__FormatMessageA@28   10005040     kernel32:KERNEL32.dll
 0002:00000044       __imp__OpenMutexA@12       10005044     kernel32:KERNEL32.dll
 0002:00000048       __imp__CreateFileMappingA@24 10005048     kernel32:KERNEL32.dll
 0002:0000004c       __imp__OpenFileMappingA@12 1000504c     kernel32:KERNEL32.dll
 0002:00000050       __imp__UnhandledExceptionFilter@4 10005050     kernel32:KERNEL32.dll
 0002:00000054       __imp__SetUnhandledExceptionFilter@4 10005054     kernel32:KERNEL32.dll
 0002:00000058       __imp__GetCurrentProcess@0 10005058     kernel32:KERNEL32.dll
 0002:0000005c       __imp__TerminateProcess@8  1000505c     kernel32:KERNEL32.dll
 0002:00000060       __imp__IsProcessorFeaturePresent@4 10005060     kernel32:KERNEL32.dll
 0002:00000064       __imp__QueryPerformanceCounter@4 10005064     kernel32:KERNEL32.dll
 0002:00000068       __imp__GetCurrentThreadId@0 10005068     kernel32:KERNEL32.dll
 0002:0000006c       __imp__GetSystemTimeAsFileTime@4 1000506c     kernel32:KERNEL32.dll
 0002:00000070       __imp__DisableThreadLibraryCalls@4 10005070     kernel32:KERNEL32.dll
 0002:00000074       __imp__InitializeSListHead@4 10005074     kernel32:KERNEL32.dll
 0002:00000078       __imp__IsDebuggerPresent@0 10005078     kernel32:KERNEL32.dll
 0002:0000007c       \177KERNEL32_NULL_THUNK_DATA 1000507c     kernel32:KERNEL32.dll
 0002:00000080       __imp__memset              10005080     vcruntime:VCRUNTIME140.dll
 0002:00000084       __imp__memcpy              10005084     vcruntime:VCRUNTIME140.dll
 0002:00000088       __imp____std_type_info_destroy_list 10005088     vcruntime:VCRUNTIME140.dll
 0002:0000008c       __imp___except_handler4_common 1000508c     vcruntime:VCRUNTIME140.dll
 0002:00000090       \177VCRUNTIME140_NULL_THUNK_DATA 10005090     vcruntime:VCRUNTIME140.dll
 0002:00000094       __imp__malloc              10005094     ucrt:api-ms-win-crt-heap-l1-1-0.dll
 0002:00000098       __imp__free                10005098     ucrt:api-ms-win-crt-heap-l1-1-0.dll
 0002:0000009c       \177api-ms-win-crt-heap-l1-1-0_NULL_THUNK_DATA 1000509c     ucrt:api-ms-win-crt-heap-l1-1-0.dll
 0002:000000a0       __imp___cexit              100050a0     ucrt:api-ms-win-crt-runtime-l1-1-0.dll
 0002:000000a4       __imp___execute_onexit_table 100050a4     ucrt:api-ms-win-crt-runtime-l1-1-0.dll
 0002:000000a8       __imp__exit                100050a8     ucrt:api-ms-win-crt-runtime-l1-1-0.dll
 0002:000000ac       __imp___initterm           100050ac     ucrt:api-ms-win-crt-runtime-l1-1-0.dll
 0002:000000b0       __imp___initterm_e         100050b0     ucrt:api-ms-win-crt-runtime-l1-1-0.dll
 0002:000000b4       __imp___seh_filter_dll     100050b4     ucrt:api-ms-win-crt-runtime-l1-1-0.dll
 0002:000000b8       __imp___configure_narrow_argv 100050b8     ucrt:api-ms-win-crt-runtime-l1-1-0.dll
 0002:000000bc       __imp___initialize_narrow_environment 100050bc     ucrt:api-ms-win-crt-runtime-l1-1-0.dll
 0002:000000c0       __imp___initialize_onexit_table 100050c0     ucrt:api-ms-win-crt-runtime-l1-1-0.dll
 0002:000000c4       \177api-ms-win-crt-runtime-l1-1-0_NULL_THUNK_DATA 100050c4     ucrt:api-ms-win-crt-runtime-l1-1-0.dll
 0002:000000c8       __imp____acrt_iob_func     100050c8     ucrt:api-ms-win-crt-stdio-l1-1-0.dll
 0002:000000cc       __imp____stdio_common_vsprintf 100050cc     ucrt:api-ms-win-crt-stdio-l1-1-0.dll
 0002:000000d0       __imp____stdio_common_vfprintf 100050d0     ucrt:api-ms-win-crt-stdio-l1-1-0.dll
 0002:000000d4       \177api-ms-win-crt-stdio-l1-1-0_NULL_THUNK_DATA 100050d4     ucrt:api-ms-win-crt-stdio-l1-1-0.dll
 0002:000000d8       __imp__strlen              100050d8     ucrt:api-ms-win-crt-string-l1-1-0.dll
 0002:000000dc       __imp__strcat              100050dc     ucrt:api-ms-win-crt-string-l1-1-0.dll
 0002:000000e0       __imp__strcpy              100050e0     ucrt:api-ms-win-crt-string-l1-1-0.dll
 0002:000000e4       \177api-ms-win-crt-string-l1-1-0_NULL_THUNK_DATA 100050e4     ucrt:api-ms-win-crt-string-l1-1-0.dll
 0002:000000e8       ___guard_check_icall_fptr  100050e8     MSVCRT:guard_support.obj
 0002:000000ec       ___xc_a                    100050ec     MSVCRT:initializers.obj
 0002:000000f0       ___xc_z                    100050f0     MSVCRT:initializers.obj
 0002:000000f4       ___xi_a                    100050f4     MSVCRT:initializers.obj
 0002:000000f8       ___xi_z                    100050f8     MSVCRT:initializers.obj
 0002:000000fc       ___xp_a                    100050fc     MSVCRT:initializers.obj
 0002:00000100       ___xp_z                    10005100     MSVCRT:initializers.obj
 0002:00000104       ___xt_a                    10005104     MSVCRT:initializers.obj
 0002:00000108       ___xt_z                    10005108     MSVCRT:initializers.obj
 0002:00000110       ??_C@_0BJ@BJPELPEK@JDWP?5header?5is?5incorrect@ 10005110     SharedMemoryConnection.obj
 0002:0000012c       ??_C@_0CD@MOHADDFA@java?1lang?1IllegalArgumentExcept@ 1000512c     SharedMemoryConnection.obj
 0002:00000150       ??_C@_0CH@FGHFIGEK@Unable?5to?5allocate?5command?5data@ 10005150     SharedMemoryConnection.obj
 0002:00000178       ??_C@_0BL@ENCPOIKC@java?1lang?1OutOfMemoryError@ 10005178     SharedMemoryConnection.obj
 0002:00000194       ??_C@_0BN@GKDBNBKE@shmemBase_receiveByte?5failed@ 10005194     SharedMemoryConnection.obj
 0002:000001b4       ??_C@_0BP@GCBMDGEM@shmemBase_receivePacket?5failed@ 100051b4     SharedMemoryConnection.obj
 0002:000001d4       ??_C@_0BK@GCMJFCKH@shmemBase_sendByte?5failed@ 100051d4     SharedMemoryConnection.obj
 0002:000001f0       ??_C@_0BM@DNIALPON@shmemBase_sendPacket?5failed@ 100051f0     SharedMemoryConnection.obj
 0002:0000020c       ??_C@_07KJFPOMFC@?$CFs?3?5?$CFs?6@ 1000520c     SharedMemoryTransport.obj
 0002:00000214       ??_C@_0BE@BGICDDI@?$CFs?0?5error?5code?5?$DN?5?$CFd@ 10005214     SharedMemoryTransport.obj
 0002:00000228       ??_C@_0BE@EBAPEBGJ@java?1io?1IOException@ 10005228     SharedMemoryTransport.obj
 0002:0000023c       ??_C@_0CL@CMFJILE@Timed?5out?5waiting?5for?5target?5VM@ 1000523c     SharedMemoryTransport.obj
 0002:00000268       ??_C@_0CO@OJENDKD@com?1sun?1jdi?1connect?1TransportTi@ 10005268     SharedMemoryTransport.obj
 0002:00000298       ??_C@_0BI@DNEMIMH@shmemBase_accept?5failed@ 10005298     SharedMemoryTransport.obj
 0002:000002b0       ??_C@_0BJ@NLGKCLLD@GetStringUTFChars?5failed@ 100052b0     SharedMemoryTransport.obj
 0002:000002cc       ??_C@_0BI@NBLNIHIB@java?1lang?1InternalError@ 100052cc     SharedMemoryTransport.obj
 0002:000002e4       ??_C@_0BI@IEJEJEDK@shmemBase_attach?5failed@ 100052e4     SharedMemoryTransport.obj
 0002:000002fc       ??_C@_0BG@COKFEFGE@shmemBase_name?5failed@ 100052fc     SharedMemoryTransport.obj
 0002:00000314       ??_C@_0BI@PCCHKLBL@Unable?5to?5create?5string@ 10005314     SharedMemoryTransport.obj
 0002:0000032c       ??_C@_0BJ@GGPEOBEL@Unable?5to?5access?5Java?5VM@ 1000532c     SharedMemoryTransport.obj
 0002:00000348       ??_C@_0CN@KCBEAAHP@Unable?5to?5initialize?5Shared?5Mem@ 10005348     SharedMemoryTransport.obj
 0002:00000378       ??_C@_0BI@BFHIKKAO@shmemBase_listen?5failed@ 10005378     SharedMemoryTransport.obj
 0002:00000390       ??_C@_02LMMGGCAJ@?3?5@     10005390     shmemBack.obj
 0002:00000394       ??_C@_0P@FPMMELAG@JDWP?9Handshake@ 10005394     shmemBack.obj
 0002:000003a4       ??_C@_0CA@FNAOCLFM@receive?5failed?5during?5handshake@ 100053a4     shmemBack.obj
 0002:000003c4       ??_C@_0DE@NCLMDMAA@handshake?5failed?5?9?5debugger?5sen@ 100053c4     shmemBack.obj
 0002:000003f8       ??_C@_0BO@DLHOCIOA@write?5failed?5during?5handshake@ 100053f8     shmemBack.obj
 0002:00000418       ??_C@_0CH@EKPBBNGK@already?5connected?5or?5already?5li@ 10005418     shmemBack.obj
 0002:00000440       ??_C@_0O@BNNCBLEN@out?5of?5memory@ 10005440     shmemBack.obj
 0002:00000450       ??_C@_0CI@DELJHAAL@failed?5to?5create?5shared?5memory?5@ 10005450     shmemBack.obj
 0002:00000478       ??_C@_0BC@DFIBIBIL@already?5connected@ 10005478     shmemBack.obj
 0002:0000048c       ??_C@_0BI@DIJAMALI@transport?5not?5listening@ 1000548c     shmemBack.obj
 0002:000004a4       ??_C@_0CB@NHHBLIIK@Timed?5out?5waiting?5for?5connectio@ 100054a4     shmemBack.obj
 0002:000004c8       ??_C@_0CK@HDEPCDBJ@failed?5to?5accept?5shared?5memory?5@ 100054c8     shmemBack.obj
 0002:000004f4       ??_C@_0BM@PMJHMKDA@Timed?5out?5waiting?5to?5attach@ 100054f4     shmemBack.obj
 0002:00000510       ??_C@_0CN@HHANKOFH@failed?5to?5attach?5to?5shared?5memo@ 10005510     shmemBack.obj
 0002:00000540       ??_C@_0P@GOGFFADL@packet?5is?5null@ 10005540     shmemBack.obj
 0002:00000550       ??_C@_0P@BHAFPBHF@invalid?5length@ 10005550     shmemBack.obj
 0002:00000560       ??_C@_0O@GLMIBBEG@not?5connected@ 10005560     shmemBack.obj
 0002:00000570       ??_C@_0BE@OGCKBGHO@write?5packet?5failed@ 10005570     shmemBack.obj
 0002:00000584       ??_C@_0BG@EJMBIBCA@receive?5packet?5failed@ 10005584     shmemBack.obj
 0002:0000059c       ??_C@_0BJ@HPOCGHOL@Other?5process?5terminated@ 1000559c     shmemBase.obj
 0002:000005b8       ??_C@_09OGKCMDDI@Timed?5out@ 100055b8     shmemBase.obj
 0002:000005c4       ??_C@_03KBEBNCEG@?4?$CFd@  100055c4     shmemBase.obj
 0002:000005c8       ??_C@_0O@KJIHJJJB@stream?5closed@ 100055c8     shmemBase.obj
 0002:000005d8       ??_C@_08KEDCEGMK@?$CFs?4mutex@ 100055d8     shmemBase.obj
 0002:000005e4       ??_C@_0L@JGHAHNJJ@?$CFs?4hasData@ 100055e4     shmemBase.obj
 0002:000005f0       ??_C@_0M@LGNPDLKN@?$CFs?4hasSpace@ 100055f0     shmemBase.obj
 0002:000005fc       ??_C@_08JJPMBCCA@?$CFs?4?$CFI64d@ 100055fc     shmemBase.obj
 0002:00000608       ??_C@_05OMNKGGE@?4ctos@    10005608     shmemBase.obj
 0002:00000610       ??_C@_05CEOPCDLH@?4stoc@   10005610     shmemBase.obj
 0002:00000618       ??_C@_0DO@DBCNLCMH@Error?3?5address?5strings?5longer?5t@ 10005618     shmemBase.obj
 0002:00000658       ??_C@_09PNEIJELD@javadebug@ 10005658     shmemBase.obj
 0002:00000664       ??_C@_09POLKDEMC@?$CFs?4accept@ 10005664     shmemBase.obj
 0002:00000670       ??_C@_09EFNMJKFA@?$CFs?4attach@ 10005670     shmemBase.obj
 0002:0000067c       ??_C@_0M@OANNIGPF@Oct?519?52022@ 1000567c     shmemBase.obj
 0002:00000688       ??_C@_0DD@MDHBMPFM@s?2src?2jdk?4jdi?2share?2native?2libd@ 10005688     shmemBase.obj
 0002:000006bc       ??_C@_0BB@DBHFCHNO@assertion?5failed@ 100056bc     shmemBase.obj
 0002:000006d0       ??_C@_0DA@JFOKPOEA@Shared?5Memory?5Transport?5?$CC?$CFs?$CC?5?$CI?$CF@ 100056d0     shmemBase.obj
 0002:00000700       ??_C@_02DKCKIIND@?$CFs@    10005700     shmemBase.obj
 0002:00000704       __pRawDllMain              10005704     MSVCRT:dll_dllmain.obj
 0002:00000704       __pDefaultRawDllMain       10005704     MSVCRT:dll_dllmain.obj
 0002:00000780       __load_config_used         10005780     MSVCRT:loadcfg.obj
 0002:00000838       ___safe_se_handler_table   10005838     <linker-defined>
 0002:00000ac4       ___rtc_iaa                 10005ac4     MSVCRT:initsect.obj
 0002:00000ac8       ___rtc_izz                 10005ac8     MSVCRT:initsect.obj
 0002:00000acc       ___rtc_taa                 10005acc     MSVCRT:initsect.obj
 0002:00000ad0       ___rtc_tzz                 10005ad0     MSVCRT:initsect.obj
 0002:00000ee8       __IMPORT_DESCRIPTOR_KERNEL32 10005ee8     kernel32:KERNEL32.dll
 0002:00000efc       __IMPORT_DESCRIPTOR_VCRUNTIME140 10005efc     vcruntime:VCRUNTIME140.dll
 0002:00000f10       __IMPORT_DESCRIPTOR_api-ms-win-crt-heap-l1-1-0 10005f10     ucrt:api-ms-win-crt-heap-l1-1-0.dll
 0002:00000f24       __IMPORT_DESCRIPTOR_api-ms-win-crt-stdio-l1-1-0 10005f24     ucrt:api-ms-win-crt-stdio-l1-1-0.dll
 0002:00000f38       __IMPORT_DESCRIPTOR_api-ms-win-crt-string-l1-1-0 10005f38     ucrt:api-ms-win-crt-string-l1-1-0.dll
 0002:00000f4c       __IMPORT_DESCRIPTOR_api-ms-win-crt-runtime-l1-1-0 10005f4c     ucrt:api-ms-win-crt-runtime-l1-1-0.dll
 0002:00000f60       __NULL_IMPORT_DESCRIPTOR   10005f60     kernel32:KERNEL32.dll
 0003:0000000c       ___security_cookie_complement 1000700c     MSVCRT:gs_cookie.obj
 0003:00000010       ___security_cookie         10007010     MSVCRT:gs_cookie.obj
 0003:00000014       ___scrt_native_dllmain_reason 10007014     MSVCRT:utility.obj
 0003:00000020       ___isa_enabled             10007020     MSVCRT:cpu_disp.obj
 0003:00000024       ___scrt_ucrt_dll_is_in_use 10007024     MSVCRT:ucrt_stubs.obj
 0003:000003a8       ?__type_info_root_node@@3U__type_info_node@@A 100073a8     MSVCRT:tncleanup.obj
 0003:000003b0       ?_OptionsStorage@?1??__local_stdio_scanf_options@@9@4_KA 100073b0     MSVCRT:default_local_stdio_options.obj
 0003:000003b8       ___scrt_current_native_startup_state 100073b8     MSVCRT:utility.obj
 0003:000003bc       ___scrt_native_startup_lock 100073bc     MSVCRT:utility.obj
 0003:000003dc       ___scrt_debugger_hook_flag 100073dc     MSVCRT:utility_desktop.obj
 0003:000003e0       ___isa_available           100073e0     MSVCRT:cpu_disp.obj
 0003:000003e4       ___favor                   100073e4     MSVCRT:cpu_disp.obj
 0003:000003e8       ?_OptionsStorage@?1??__local_stdio_printf_options@@9@9 100073e8     <common>
 0003:000003f0       ___dyn_tls_init_callback   100073f0     <common>

 entry point at        0001:00002730

 Static symbols

 0000:ffff6000       .debug$S                   10000000     dt_shmem.exp
 0000:ffff6000       .debug$S                   10000000     vcruntime:VCRUNTIME140.dll
 0000:ffff6000       .debug$S                   10000000     vcruntime:VCRUNTIME140.dll
 0000:ffff6000       .debug$S                   10000000     vcruntime:VCRUNTIME140.dll
 0000:ffff6000       .debug$S                   10000000     vcruntime:VCRUNTIME140.dll
 0000:ffff6000       .debug$S                   10000000     vcruntime:VCRUNTIME140.dll
 0000:ffff6000       .debug$S                   10000000     vcruntime:VCRUNTIME140.dll
 0000:ffff6000       .debug$S                   10000000     ucrt:api-ms-win-crt-heap-l1-1-0.dll
 0000:ffff6000       .debug$S                   10000000     ucrt:api-ms-win-crt-heap-l1-1-0.dll
 0000:ffff6000       .debug$S                   10000000     ucrt:api-ms-win-crt-runtime-l1-1-0.dll
 0000:ffff6000       .debug$S                   10000000     ucrt:api-ms-win-crt-runtime-l1-1-0.dll
 0000:ffff6000       .debug$S                   10000000     ucrt:api-ms-win-crt-runtime-l1-1-0.dll
 0000:ffff6000       .debug$S                   10000000     ucrt:api-ms-win-crt-runtime-l1-1-0.dll
 0000:ffff6000       .debug$S                   10000000     ucrt:api-ms-win-crt-runtime-l1-1-0.dll
 0000:ffff6000       .debug$S                   10000000     ucrt:api-ms-win-crt-runtime-l1-1-0.dll
 0000:ffff6000       .debug$S                   10000000     ucrt:api-ms-win-crt-runtime-l1-1-0.dll
 0000:ffff6000       .debug$S                   10000000     ucrt:api-ms-win-crt-runtime-l1-1-0.dll
 0000:ffff6000       .debug$S                   10000000     ucrt:api-ms-win-crt-runtime-l1-1-0.dll
 0000:ffff6000       .debug$S                   10000000     ucrt:api-ms-win-crt-runtime-l1-1-0.dll
 0000:ffff6000       .debug$S                   10000000     ucrt:api-ms-win-crt-runtime-l1-1-0.dll
 0000:ffff6000       .debug$S                   10000000     ucrt:api-ms-win-crt-runtime-l1-1-0.dll
 0000:ffff6000       .debug$S                   10000000     ucrt:api-ms-win-crt-runtime-l1-1-0.dll
 0000:ffff6000       .debug$S                   10000000     ucrt:api-ms-win-crt-stdio-l1-1-0.dll
 0000:ffff6000       .debug$S                   10000000     ucrt:api-ms-win-crt-stdio-l1-1-0.dll
 0000:ffff6000       .debug$S                   10000000     ucrt:api-ms-win-crt-stdio-l1-1-0.dll
 0000:ffff6000       .debug$S                   10000000     ucrt:api-ms-win-crt-string-l1-1-0.dll
 0000:ffff6000       .debug$S                   10000000     ucrt:api-ms-win-crt-string-l1-1-0.dll
 0000:ffff6000       .debug$S                   10000000     ucrt:api-ms-win-crt-string-l1-1-0.dll
 0000:ffff6000       .debug$S                   10000000     kernel32:KERNEL32.dll
 0000:ffff6000       .debug$S                   10000000     kernel32:KERNEL32.dll
 0000:ffff6000       .debug$S                   10000000     kernel32:KERNEL32.dll
 0000:ffff6000       .debug$S                   10000000     kernel32:KERNEL32.dll
 0000:ffff6000       .debug$S                   10000000     kernel32:KERNEL32.dll
 0000:ffff6000       .debug$S                   10000000     kernel32:KERNEL32.dll
 0000:ffff6000       .debug$S                   10000000     kernel32:KERNEL32.dll
 0000:ffff6000       .debug$S                   10000000     kernel32:KERNEL32.dll
 0000:ffff6000       .debug$S                   10000000     kernel32:KERNEL32.dll
 0000:ffff6000       .debug$S                   10000000     kernel32:KERNEL32.dll
 0000:ffff6000       .debug$S                   10000000     kernel32:KERNEL32.dll
 0000:ffff6000       .debug$S                   10000000     kernel32:KERNEL32.dll
 0000:ffff6000       .debug$S                   10000000     kernel32:KERNEL32.dll
 0000:ffff6000       .debug$S                   10000000     kernel32:KERNEL32.dll
 0000:ffff6000       .debug$S                   10000000     kernel32:KERNEL32.dll
 0000:ffff6000       .debug$S                   10000000     kernel32:KERNEL32.dll
 0000:ffff6000       .debug$S                   10000000     kernel32:KERNEL32.dll
 0000:ffff6000       .debug$S                   10000000     kernel32:KERNEL32.dll
 0000:ffff6000       .debug$S                   10000000     kernel32:KERNEL32.dll
 0000:ffff6000       .debug$S                   10000000     kernel32:KERNEL32.dll
 0000:ffff6000       .debug$S                   10000000     kernel32:KERNEL32.dll
 0000:ffff6000       .debug$S                   10000000     kernel32:KERNEL32.dll
 0000:ffff6000       .debug$S                   10000000     kernel32:KERNEL32.dll
 0000:ffff6000       .debug$S                   10000000     kernel32:KERNEL32.dll
 0000:ffff6000       .debug$S                   10000000     kernel32:KERNEL32.dll
 0000:ffff6000       .debug$S                   10000000     kernel32:KERNEL32.dll
 0000:ffff6000       .debug$S                   10000000     kernel32:KERNEL32.dll
 0000:ffff6000       .debug$S                   10000000     kernel32:KERNEL32.dll
 0000:ffff6000       .debug$S                   10000000     kernel32:KERNEL32.dll
 0000:ffff6000       .debug$S                   10000000     kernel32:KERNEL32.dll
 0000:ffff6000       .debug$S                   10000000     kernel32:KERNEL32.dll
 0000:ffff6000       .debug$S                   10000000     kernel32:KERNEL32.dll
 0000:ffff6000       .debug$S                   10000000     kernel32:KERNEL32.dll
 0000:ffff6000       .debug$S                   10000000     kernel32:KERNEL32.dll
 0001:00000116       _byteArrayToPacket         10001116 f   SharedMemoryConnection.obj
 0001:00000257       _intToBigInt               10001257 f   SharedMemoryConnection.obj
 0001:00000293       _isBigEndian               10001293 f   SharedMemoryConnection.obj
 0001:000002b4       _packetToByteArray         100012b4 f   SharedMemoryConnection.obj
 0001:000003bb       _allocateWrapper           100013bb f   SharedMemoryTransport.obj
 0001:000006bc       _handshake                 100016bc f   shmemBack.obj
 0001:00000819       _setLastError              10001819 f   shmemBack.obj
 0001:00000910       _shmemAccept@20            10001910 f   shmemBack.obj
 0001:00000994       _shmemAttach@24            10001994 f   shmemBack.obj
 0001:00000a23       _shmemClose@4              10001a23 f   shmemBack.obj
 0001:00000a3f       _shmemGetCapabilities@8    10001a3f f   shmemBack.obj
 0001:00000a67       _shmemGetLastError@8       10001a67 f   shmemBack.obj
 0001:00000ab0       _shmemIsOpen@4             10001ab0 f   shmemBack.obj
 0001:00000abd       _shmemReadPacket@8         10001abd f   shmemBack.obj
 0001:00000b15       _shmemStartListening@12    10001b15 f   shmemBack.obj
 0001:00000bb8       _shmemStopListening@4      10001bb8 f   shmemBack.obj
 0001:00000bd4       _shmemWritePacket@8        10001bd4 f   shmemBack.obj
 0001:00000c5b       _allocConnection           10001c5b f   shmemBase.obj
 0001:00000c8c       _clearLastError            10001c8c f   shmemBase.obj
 0001:00000cb6       _closeConnection           10001cb6 f   shmemBase.obj
 0001:00000d47       _closeStream               10001d47 f   shmemBase.obj
 0001:00000e33       _closeTransport            10001e33 f   shmemBase.obj
 0001:00000e69       _createConnection          10001e69 f   shmemBase.obj
 0001:00000fcd       _createEvent               10001fcd f   shmemBase.obj
 0001:00000fe0       _createMutex               10001fe0 f   shmemBase.obj
 0001:00000fe5       _createSharedMem           10001fe5 f   shmemBase.obj
 0001:00001000       _createStream              10002000 f   shmemBase.obj
 0001:0000110a       _createTransport           1000210a f   shmemBase.obj
 0001:000012d3       _createWithGeneratedName   100022d3 f   shmemBase.obj
 0001:00001369       _doAttach                  10002369 f   shmemBase.obj
 0001:000013b7       _enterMutex                100023b7 f   shmemBase.obj
 0001:000014bd       _openConnection            100024bd f   shmemBase.obj
 0001:000015a4       _openStream                100025a4 f   shmemBase.obj
 0001:00001632       _openTransport             10002632 f   shmemBase.obj
 0001:00001744       _receiveBytes              10002744 f   shmemBase.obj
 0001:00001845       _sendBytes                 10002845 f   shmemBase.obj
 0001:0000194c       _setLastError              1000294c f   shmemBase.obj
 0001:000019b6       _setLastErrorMsg           100029b6 f   shmemBase.obj
 0001:00001c1b       _shmemBase_receiveByte_internal 10002c1b f   shmemBase.obj
 0001:00001cf0       _shmemBase_receivePacket_internal 10002cf0 f   shmemBase.obj
 0001:00001e23       _shmemBase_sendByte_internal 10002e23 f   shmemBase.obj
 0001:00001efe       _shmemBase_sendPacket_internal 10002efe f   shmemBase.obj
 0001:00001ff3       _waitForData               10002ff3 f   shmemBase.obj
 0001:0000206b       _waitForSpace              1000306b f   shmemBase.obj
 0001:000023f0       ?dllmain_crt_dispatch@@YGHQAUHINSTANCE__@@KQAX@Z 100033f0 f   MSVCRT:dll_dllmain.obj
 0001:00002443       ?dllmain_crt_process_attach@@YAHQAUHINSTANCE__@@QAX@Z 10003443 f   MSVCRT:dll_dllmain.obj
 0001:0000254a       ?dllmain_crt_process_detach@@YAH_N@Z 1000354a f   MSVCRT:dll_dllmain.obj
 0001:000025fa       ?dllmain_dispatch@@YAHQAUHINSTANCE__@@KQAX@Z 100035fa f   MSVCRT:dll_dllmain.obj
 0001:00002705       ?dllmain_raw@@YGHQAUHINSTANCE__@@KQAX@Z 10003705 f   MSVCRT:dll_dllmain.obj
 0001:00002874       ___get_entropy             10003874 f   MSVCRT:gs_support.obj
 0001:00002969       ?find_pe_section@@YAPAU_IMAGE_SECTION_HEADER@@QAEI@Z 10003969 f   MSVCRT:utility.obj
 0001:00002dd0       $$000000                   10003dd0     MSVCRT:sehprolg4.obj
 0002:00000708       _GS_ExceptionPointers      10005708     MSVCRT:gs_report.obj
 0002:00000ad8       __sehtable$?dllmain_crt_process_attach@@YAHQAUHINSTANCE__@@QAX@Z 10005ad8     MSVCRT:dll_dllmain.obj
 0002:00000af8       __sehtable$?dllmain_crt_process_detach@@YAH_N@Z 10005af8     MSVCRT:dll_dllmain.obj
 0002:00000b20       __sehtable$?dllmain_dispatch@@YAHQAUHINSTANCE__@@KQAX@Z 10005b20     MSVCRT:dll_dllmain.obj
 0002:00000b40       __sehtable$___scrt_is_nonwritable_in_current_image 10005b40     MSVCRT:utility.obj
 0002:00000b60       .edata                     10005b60     dt_shmem.exp
 0002:00000b88       rgpv                       10005b88     dt_shmem.exp
 0002:00000bb8       rgszName                   10005bb8     dt_shmem.exp
 0002:00000be8       rgwOrd                     10005be8     dt_shmem.exp
 0002:00000c00       szName                     10005c00     dt_shmem.exp
 0002:00000c0d       $N00001                    10005c0d     dt_shmem.exp
 0002:00000c46       $N00002                    10005c46     dt_shmem.exp
 0002:00000c85       $N00003                    10005c85     dt_shmem.exp
 0002:00000cc6       $N00004                    10005cc6     dt_shmem.exp
 0002:00000d02       $N00005                    10005d02     dt_shmem.exp
 0002:00000d40       $N00006                    10005d40     dt_shmem.exp
 0002:00000d80       $N00007                    10005d80     dt_shmem.exp
 0002:00000dc0       $N00008                    10005dc0     dt_shmem.exp
 0002:00000e02       $N00009                    10005e02     dt_shmem.exp
 0002:00000e3f       $N00010                    10005e3f     dt_shmem.exp
 0002:00000e87       $N00011                    10005e87     dt_shmem.exp
 0002:00000ece       $N00012                    10005ece     dt_shmem.exp
 0002:000012ac       .idata$6                   100062ac     kernel32:KERNEL32.dll
 0002:00001308       .idata$6                   10006308     vcruntime:VCRUNTIME140.dll
 0002:0000143e       .idata$6                   1000643e     ucrt:api-ms-win-crt-heap-l1-1-0.dll
 0002:0000145e       .idata$6                   1000645e     ucrt:api-ms-win-crt-stdio-l1-1-0.dll
 0002:0000147e       .idata$6                   1000647e     ucrt:api-ms-win-crt-string-l1-1-0.dll
 0002:000014a0       .idata$6                   100064a0     ucrt:api-ms-win-crt-runtime-l1-1-0.dll
 0003:00000000       _callbacks                 10007000     SharedMemoryTransport.obj
 0003:00000008       _single_env                10007008     shmemBack.obj
 0003:00000028       _byte_ordering_known       10007028     SharedMemoryConnection.obj
 0003:0000002c       _is_big_endian             1000702c     SharedMemoryConnection.obj
 0003:00000030       _interface                 10007030     shmemBack.obj
 0003:00000060       _transport                 10007060     shmemBack.obj
 0003:00000064       _connection                10007064     shmemBack.obj
 0003:00000068       _callbacks                 10007068     shmemBack.obj
 0003:0000006c       _initialized               1000706c     shmemBack.obj
 0003:00000070       _tlsIndex                  10007070     shmemBack.obj
 0003:00000074       _callback                  10007074     shmemBase.obj
 0003:00000078       _jvm                       10007078     shmemBase.obj
 0003:0000007c       _tlsIndex                  1000707c     shmemBase.obj
 0003:00000080       ?__proc_attached@@3HA      10007080     MSVCRT:dll_dllmain.obj
 0003:00000088       _GS_ExceptionRecord        10007088     MSVCRT:gs_report.obj
 0003:000000d8       _GS_ContextRecord          100070d8     MSVCRT:gs_report.obj
 0003:000003c0       ?is_initialized_as_dll@@3_NA 100073c0     MSVCRT:utility.obj
 0003:000003c1       ?module_local_atexit_table_initialized@@3_NA 100073c1     MSVCRT:utility.obj
 0003:000003c4       ?module_local_atexit_table@@3U_onexit_table_t@@A 100073c4     MSVCRT:utility.obj
 0003:000003d0       ?module_local_at_quick_exit_table@@3U_onexit_table_t@@A 100073d0     MSVCRT:utility.obj
 0004:00000060       $R000000                   10008060     dt_shmem.dll.res
